:1000000012C0189518951895189518951895189563
:100010001895189518951895189518951895189578
:100020001895189518958FED8DBFC0ECE8EB4E2E06
:10003000DD275D2EEEE7F0E0A0E6B0E0A89584B7FE
:10004000082E877F84BF88E1992781BD91BD8827CD
:100050008D933197E9F783E389B980E082B988E12C
:100060008AB966248FEF87BB8FEF81BB80E088BBA6
:10007000929A939A949AA3E6E4E7F2E0CFD0A5E6A9
:10008000E4E7F2E0CBD0A7E6E4E7F2E0C7D0A6D001
:10009000A1E68D9388278C93A1E6E6E7F2E0D7D01E
:1000A00009F005C09FD0A3E68D9388278C93A1E625
:1000B000E8E7F2E0CCD009F005C094D0A5E68D9336
:1000C00088278C93A1E6EAE7F2E0C1D009F005C0E9
:1000D00089D0A7E68D9388278C9380E088BB95987C
:1000E0009698929A9498A3E68C91A9E68C93A9E6A7
:1000F0008C9180538C9300916900083008F008C0FF
:10010000A9E68C91A8E39DD092D09C91982B9C93CA
:1001100000916900083009F001C0959A00916900CA
:10012000093009F001C0969A85E090E068D080E03F
:1001300088BB95989698949A9398A5E68C91A9E691
:100140008C93A9E68C9180538C93009169000830C0
:1001500008F008C0A9E68C91A8E373D068D09C9100
:10016000982B9C9300916900083009F001C0959A82
:1001700000916900093009F001C0969A85E090E08D
:100180003ED080E088BB95989698939A9298A7E67F
:100190008C91A9E68C93A9E68C9180538C93009165
:1001A0006900083008F008C0A9E68C91A8E349D09E
:1001B0003ED09C91982B9C9300916900083009F0E7
:1001C00001C0959A00916900093009F001C0969A22
:1001D00085E090E014D05BCFF894FFCF88275F9B39
:1001E000089500C05F9BFECF8CB108953197F1F761
:1001F0000895689462F80895E89462F80895EF937A
:10020000FF93EE27E82BE92B31F0E0EDF7E0319793
:10021000F1F70197D1F7FF91EF91089504D00D9276
:100220000020E1F70895C89531960020089591E0E7
:10023000882321F08894991F8A95E9F7892F909552
:100240000895883018F011968850FBCF089568946F
:1002500001C0E894AF93BF938D9116F0919102C0C5
:10026000E2DF902D891718F011F48823A9F7BF91C8
:0C027000AF91089530006100620063004F
:00000001FF
